################################################################################
#                                                                              #
#      IAR Universal Linker V4.60I/386                                         #
#                                                                              #
#           Link time     =  14/May/2008  12:49:24                             #
#           Target CPU    =  ARM                                               #
#           List file     =  D:\Pasha\elf\googlecode\MyMenu2\MyMenu2_Editor\Re #
#                            lease\List\MyMenu2_Editor.map                     #
#           Output file 1 =  D:\Pasha\elf\googlecode\MyMenu2\MyMenu2_Editor\Re #
#                            lease\Exe\MyMenu2_Editor.elf                      #
#                            Format: elf, variant: -ynpra                      #
#           Command line  =  D:\Pasha\elf\googlecode\MyMenu2\MyMenu2_Editor\Re #
#                            lease\Obj\ed_gui.r79                              #
#                            D:\Pasha\elf\googlecode\MyMenu2\MyMenu2_Editor\Re #
#                            lease\Obj\func.r79                                #
#                            D:\Pasha\elf\googlecode\MyMenu2\MyMenu2_Editor\Re #
#                            lease\Obj\main.r79                                #
#                            D:\Pasha\elf\googlecode\MyMenu2\MyMenu2_Editor\Re #
#                            lease\Obj\open_select_file.r79                    #
#                            D:\Pasha\elf\googlecode\MyMenu2\MyMenu2_Editor\Re #
#                            lease\Obj\option_menu.r79                         #
#                            -o                                                #
#                            D:\Pasha\elf\googlecode\MyMenu2\MyMenu2_Editor\Re #
#                            lease\Exe\MyMenu2_Editor.elf                      #
#                            -Felf -l                                          #
#                            D:\Pasha\elf\googlecode\MyMenu2\MyMenu2_Editor\Re #
#                            lease\List\MyMenu2_Editor.map                     #
#                            -xmsnio -f                                        #
#                            D:\Pasha\elf\googlecode\MyMenu2\MyMenu2_Editor\.. #
#                            \test.xcl                                         #
#                            (-carm -V(CODE)CODE_AREA,12                       #
#                            -V(DATA)DATA_AREA,12                              #
#                            -Z(CODE_AREA)ELFBEGIN,DATA_ID,START,CODE,DATA_C,I #
#                            NITTAB,DATA_Z,DATA_N,MYSEG,CONFIG_C=0-FFFFFFFF    #
#                            -Z(DATA_AREA)DATA_I=0-FFFFFFFF) -ynpra            #
#                            "D:\Pasha\Embedded Workbench 4.0 Evaluation2\ARM\ #
#                            LIB\dl5tpainl8n.r79"                              #
#                            -s main                                           #
#                                                                              #
#                        Copyright 1987-2007 IAR Systems. All rights reserved. #
################################################################################





                ****************************************
                *                                      *
                *           CROSS REFERENCE            *
                *                                      *
                ****************************************

       Program entry at : CODE_AREA 00000D78  Relocatable, from module : main




                ****************************************
                *                                      *
                *            RUNTIME MODEL             *
                *                                      *
                ****************************************

  StackAlign4  = USED
  __cpu_mode   = __pcs__interwork
  __data_model = absolute
  __endian     = little
  __rt_version = 6



                ****************************************
                *                                      *
                *              MODULE MAP              *
                *                                      *
                ****************************************


  DEFINED ABSOLUTE ENTRIES
    *************************************************************************

  DEFINED ABSOLUTE ENTRIES
    *************************************************************************

  FILE NAME : D:\Pasha\elf\googlecode\MyMenu2\MyMenu2_Editor\Release\Obj\ed_gui.r79
  PROGRAM MODULE, NAME : ed_gui

  SEGMENTS IN THE MODULE
  ======================
DATA_C
  Relative segment, address: CODE_AREA 00001928 - 0000192F (0x8 bytes), align: 2
  Segment part 2.             Intra module refs:   edheader
    -------------------------------------------------------------------------
DATA_C
  Relative segment, address: CODE_AREA 00001930 - 0000194B (0x1c bytes), align: 2
  Segment part 3.             Intra module refs:   on_exmenu
    -------------------------------------------------------------------------
DATA_C
  Segment part 4. NOT NEEDED.
    -------------------------------------------------------------------------
DATA_C
  Relative segment, address: CODE_AREA 0000194C - 0000196F (0x24 bytes), align: 2
  Segment part 5.             Intra module refs:   edit_ml
           ENTRY                   ADDRESS         REF BY
           =====                   =======         ======
           edheader                0000194C 
    -------------------------------------------------------------------------
DATA_C
  Relative segment, address: CODE_AREA 00001970 - 00001987 (0x18 bytes), align: 2
  Segment part 6.             Intra module refs:   ed_skt
           ENTRY                   ADDRESS         REF BY
           =====                   =======         ======
           ed_sk                   00001970 
    -------------------------------------------------------------------------
DATA_C
  Relative segment, address: CODE_AREA 00001988 - 0000198F (0x8 bytes), align: 2
  Segment part 7.             Intra module refs:   Segment part 9
           ENTRY                   ADDRESS         REF BY
           =====                   =======         ======
           ed_skt                  00001988 
    -------------------------------------------------------------------------
CODE
  Segment part 10. NOT NEEDED.
    -------------------------------------------------------------------------
CODE
  Relative segment, address: CODE_AREA 00000124 - 00000193 (0x70 bytes), align: 2
  Segment part 11.            Intra module refs:   ed_onkey
           ENTRY                   ADDRESS         REF BY
           =====                   =======         ======
           on_exmenu               00000124 
               stack 1 = 00000000 ( 00000008 )
    -------------------------------------------------------------------------
CODE
  Segment part 12. NOT NEEDED.
    -------------------------------------------------------------------------
CODE
  Relative segment, address: CODE_AREA 00000194 - 000001F3 (0x60 bytes), align: 2
  Segment part 13.            Intra module refs:   Segment part 9
           ENTRY                   ADDRESS         REF BY
           =====                   =======         ======
           ed_onkey                00000194 
               stack 1 = 00000000 ( 0000000C )
    -------------------------------------------------------------------------
CODE
  Segment part 14. NOT NEEDED.
    -------------------------------------------------------------------------
CODE
  Relative segment, address: CODE_AREA 000001F4 - 00000267 (0x74 bytes), align: 2
  Segment part 15.            Intra module refs:   Segment part 9
           ENTRY                   ADDRESS         REF BY
           =====                   =======         ======
           ed_ghook                000001F4 
               stack 1 = 00000000 ( 00000034 )
    -------------------------------------------------------------------------
CODE
  Segment part 16. NOT NEEDED.
    -------------------------------------------------------------------------
CODE
  Relative segment, address: CODE_AREA 00000268 - 0000026B (0x4 bytes), align: 2
  Segment part 17.            Intra module refs:   Segment part 9
           ENTRY                   ADDRESS         REF BY
           =====                   =======         ======
           ed_locret               00000268 
    -------------------------------------------------------------------------
CODE
  Segment part 18. NOT NEEDED.
    -------------------------------------------------------------------------
DATA_I
  Relative segment, address: DATA_AREA 00000000 - 00000037 (0x38 bytes), align: 2
  Segment part 8.             Intra module refs:   edit_ml
           ENTRY                   ADDRESS         REF BY
           =====                   =======         ======
           ed_desc                 00000000 
    -------------------------------------------------------------------------
CODE
  Relative segment, address: CODE_AREA 0000026C - 0000048F (0x224 bytes), align: 2
  Segment part 19.
           ENTRY                   ADDRESS         REF BY
           =====                   =======         ======
           edit_ml                 0000026C        menu_add (option_menu)
                                                   menu_edit (option_menu)
                                                   menu_insert (option_menu)
                                                   menu_onkey (main)
               stack 1 = 00000000 ( 00000060 )
    -------------------------------------------------------------------------
CODE
  Segment part 20. NOT NEEDED.Intra module refs:   on_exmenu
    -------------------------------------------------------------------------
CSTACK
  Segment part 1. NOT NEEDED.
    -------------------------------------------------------------------------
DATA_ID
  Relative segment, address: CODE_AREA 00000000 - 00000037 (0x38 bytes), align: 2
  Segment part 9.             Intra module refs:   ed_desc
    -------------------------------------------------------------------------
DATA_ID
  Segment part 21. NOT NEEDED.
           ENTRY                   ADDRESS         REF BY
           =====                   =======         ======
           ?*?DATA_ID              
    -------------------------------------------------------------------------
INITTAB
  Relative segment, address: CODE_AREA 00001D70 - 00001D7B (0xc bytes), align: 2
  Segment part 22. ROOT.
           ENTRY                   ADDRESS         REF BY
           =====                   =======         ======
           ?init?tab?DATA_I        00001D70 

    *************************************************************************

  FILE NAME : D:\Pasha\elf\googlecode\MyMenu2\MyMenu2_Editor\Release\Obj\func.r79
  PROGRAM MODULE, NAME : func

  SEGMENTS IN THE MODULE
  ======================
ELFBEGIN
  Relative segment, address: CODE_AREA 00000000, align: 0
  Segment part 0. ROOT.
           ENTRY                   ADDRESS         REF BY
           =====                   =======         ======
           ELF_BEGIN               00000000        Killer (main)
    -------------------------------------------------------------------------
CODE
  Relative segment, address: CODE_AREA 00000490 - 00000497 (0x8 bytes), align: 2
  Segment part 1. ROOT.
           ENTRY                   ADDRESS         REF BY
           =====                   =======         ======
           kill_data               00000490        Killer (main)
           seqkill                 00000494 

    *************************************************************************

  FILE NAME : D:\Pasha\elf\googlecode\MyMenu2\MyMenu2_Editor\Release\Obj\main.r79
  PROGRAM MODULE, NAME : main

  SEGMENTS IN THE MODULE
  ======================
DATA_Z
  Relative segment, address: CODE_AREA 00001D88 - 00001DA7 (0x20 bytes), align: 2
  Segment part 10.            Intra module refs:   Segment part 25
                                                   Segment part 50
                                                   Segment part 53
                                                   menu_onkey
           ENTRY                   ADDRESS         REF BY
           =====                   =======         ======
           EDGUI_ID                00001D90        edit_ml (ed_gui)
           MAIN_GUI_ID             00001D94        Segment part 36 (option_menu)
           buf                     00001D88 
           menu_item_n             00001D98        Segment part 29 (option_menu)
           ml_edit_tmp             00001DA4        Segment part 34 (option_menu)
                                                   edit_ml (ed_gui)
           mltop                   00001D8C        Segment part 35 (option_menu)
           ws_edit_functmp         00001DA0        ed_ghook (ed_gui)
           ws_edit_nametmp         00001D9C        ed_ghook (ed_gui)
    -------------------------------------------------------------------------
CODE
  Segment part 17. NOT NEEDED.
    -------------------------------------------------------------------------
CODE
  Segment part 18. NOT NEEDED.
           ENTRY                   ADDRESS         REF BY
           =====                   =======         ======
           utf8_2str               
               not allocated function
    -------------------------------------------------------------------------
CODE
  Segment part 19. NOT NEEDED.
    -------------------------------------------------------------------------
CODE
  Relative segment, address: CODE_AREA 00000498 - 0000051B (0x84 bytes), align: 2
  Segment part 20.            Intra module refs:   read_cfg
           ENTRY                   ADDRESS         REF BY
           =====                   =======         ======
           AddtoMenuList           00000498 
               stack 1 = 00000000 ( 0000001C )
    -------------------------------------------------------------------------
CODE
  Segment part 21. NOT NEEDED.
    -------------------------------------------------------------------------
CODE
  Relative segment, address: CODE_AREA 0000051C - 00000563 (0x48 bytes), align: 2
  Segment part 22.            Intra module refs:   Killer
                                                   read_cfg
           ENTRY                   ADDRESS         REF BY
           =====                   =======         ======
           FreeMenuList            0000051C 
               stack 1 = 00000000 ( 0000000C )
    -------------------------------------------------------------------------
CODE
  Segment part 23. NOT NEEDED.
    -------------------------------------------------------------------------
CODE
  Relative segment, address: CODE_AREA 00000564 - 0000059B (0x38 bytes), align: 2
  Segment part 24.            Intra module refs:   menu_iconhndl
                                                   menu_onkey
           ENTRY                   ADDRESS         REF BY
           =====                   =======         ======
           get_mlitem              00000564 
    -------------------------------------------------------------------------
CODE
  Relative segment, address: CODE_AREA 0000059C - 0000059F (0x4 bytes), align: 2
  Segment part 25.            Intra module refs:   FreeMenuList
                                                   get_mlitem
    -------------------------------------------------------------------------
CODE
  Segment part 26. NOT NEEDED.
    -------------------------------------------------------------------------
CODE
  Relative segment, address: CODE_AREA 000005A0 - 000005CF (0x30 bytes), align: 2
  Segment part 27.            Intra module refs:   read_cfg
           ENTRY                   ADDRESS         REF BY
           =====                   =======         ======
           strchrinline            000005A0 
    -------------------------------------------------------------------------
CODE
  Segment part 28. NOT NEEDED.
    -------------------------------------------------------------------------
CODE
  Relative segment, address: CODE_AREA 000005D0 - 000005EF (0x20 bytes), align: 2
  Segment part 29.            Intra module refs:   read_cfg
           ENTRY                   ADDRESS         REF BY
           =====                   =======         ======
           gotoRealPos             000005D0 
    -------------------------------------------------------------------------
CODE
  Segment part 30. NOT NEEDED.
    -------------------------------------------------------------------------
CODE
  Relative segment, address: CODE_AREA 000005F0 - 0000060F (0x20 bytes), align: 2
  Segment part 31.            Intra module refs:   CheckType
                                                   read_cfg
           ENTRY                   ADDRESS         REF BY
           =====                   =======         ======
           gotoLineEnd             000005F0 
    -------------------------------------------------------------------------
CODE
  Segment part 32. NOT NEEDED.
    -------------------------------------------------------------------------
CODE
  Relative segment, address: CODE_AREA 00000610 - 0000066B (0x5c bytes), align: 2
  Segment part 33.            Intra module refs:   read_cfg
                                                   save_ml
           ENTRY                   ADDRESS         REF BY
           =====                   =======         ======
           CheckType               00000610 
               stack 1 = 00000000 ( 00000004 )
    -------------------------------------------------------------------------
CODE
  Segment part 34. NOT NEEDED.
    -------------------------------------------------------------------------
CODE
  Relative segment, address: CODE_AREA 0000066C - 00000887 (0x21c bytes), align: 2
  Segment part 35.            Intra module refs:   maincsm_oncreate
           ENTRY                   ADDRESS         REF BY
           =====                   =======         ======
           read_cfg                0000066C 
               stack 1 = 00000000 ( 00000048 )
    -------------------------------------------------------------------------
CODE
  Segment part 36. NOT NEEDED.
    -------------------------------------------------------------------------
CODE
  Relative segment, address: CODE_AREA 00000888 - 000009B3 (0x12c bytes), align: 2
  Segment part 37.            Intra module refs:   save_ml
           ENTRY                   ADDRESS         REF BY
           =====                   =======         ======
           save_file               00000888        menu_del (option_menu)
                                                   menu_movedown (option_menu)
                                                   menu_moveup (option_menu)
               stack 1 = 00000000 ( 00000118 )
    -------------------------------------------------------------------------
CODE
  Segment part 38. NOT NEEDED.
    -------------------------------------------------------------------------
CODE
  Relative segment, address: CODE_AREA 000009B4 - 00000A7B (0xc8 bytes), align: 2
  Segment part 39.            Intra module refs:   maincsm_onmessage
           ENTRY                   ADDRESS         REF BY
           =====                   =======         ======
           save_ml                 000009B4 
               stack 1 = 00000000 ( 00000014 )
    -------------------------------------------------------------------------
CODE
  Segment part 40. NOT NEEDED.
    -------------------------------------------------------------------------
CODE
  Relative segment, address: CODE_AREA 00000A7C - 00000B47 (0xcc bytes), align: 2
  Segment part 41.            Intra module refs:   Segment part 14
           ENTRY                   ADDRESS         REF BY
           =====                   =======         ======
           menu_onkey              00000A7C 
               stack 1 = 00000000 ( 00000008 )
    -------------------------------------------------------------------------
CODE
  Segment part 42. NOT NEEDED.
    -------------------------------------------------------------------------
CODE
  Relative segment, address: CODE_AREA 00000B48 - 00000B5B (0x14 bytes), align: 2
  Segment part 43.            Intra module refs:   Segment part 14
           ENTRY                   ADDRESS         REF BY
           =====                   =======         ======
           menu_ghook              00000B48 
               stack 1 = 00000000 ( 00000004 )
    -------------------------------------------------------------------------
CODE
  Segment part 44. NOT NEEDED.
    -------------------------------------------------------------------------
CODE
  Relative segment, address: CODE_AREA 00000B5C - 00000BDF (0x84 bytes), align: 2
  Segment part 45.            Intra module refs:   Segment part 14
           ENTRY                   ADDRESS         REF BY
           =====                   =======         ======
           menu_iconhndl           00000B5C 
               stack 1 = 00000000 ( 00000018 )
    -------------------------------------------------------------------------
CODE
  Segment part 46. NOT NEEDED.
    -------------------------------------------------------------------------
CODE
  Relative segment, address: CODE_AREA 00000BE0 - 00000C7F (0xa0 bytes), align: 2
  Segment part 47.            Intra module refs:   MAINCSM
           ENTRY                   ADDRESS         REF BY
           =====                   =======         ======
           maincsm_oncreate        00000BE0 
               stack 1 = 00000000 ( 00000020 )
    -------------------------------------------------------------------------
CODE
  Segment part 48. NOT NEEDED.
    -------------------------------------------------------------------------
CODE
  Relative segment, address: CODE_AREA 00000C80 - 00000D03 (0x84 bytes), align: 2
  Segment part 49.            Intra module refs:   MAINCSM
           ENTRY                   ADDRESS         REF BY
           =====                   =======         ======
           maincsm_onmessage       00000C80 
               stack 1 = 00000000 ( 0000000C )
    -------------------------------------------------------------------------
CODE
  Relative segment, address: CODE_AREA 00000D04 - 00000D07 (0x4 bytes), align: 2
  Segment part 50.            Intra module refs:   AddtoMenuList
                                                   maincsm_onmessage
                                                   save_file
                                                   save_ml
    -------------------------------------------------------------------------
CODE
  Segment part 51. NOT NEEDED.
    -------------------------------------------------------------------------
CODE
  Relative segment, address: CODE_AREA 00000D08 - 00000D43 (0x3c bytes), align: 2
  Segment part 52.            Intra module refs:   maincsm_onclose
           ENTRY                   ADDRESS         REF BY
           =====                   =======         ======
           Killer                  00000D08 
               stack 1 = 00000000 ( 00000008 )
    -------------------------------------------------------------------------
CODE
  Relative segment, address: CODE_AREA 00000D44 - 00000D47 (0x4 bytes), align: 2
  Segment part 53.            Intra module refs:   Killer
                                                   maincsm_oncreate
                                                   read_cfg
    -------------------------------------------------------------------------
CODE
  Segment part 54. NOT NEEDED.
    -------------------------------------------------------------------------
CODE
  Relative segment, address: CODE_AREA 00000D48 - 00000D5B (0x14 bytes), align: 2
  Segment part 55.            Intra module refs:   MAINCSM
           ENTRY                   ADDRESS         REF BY
           =====                   =======         ======
           maincsm_onclose         00000D48 
               stack 1 = 00000000 ( 00000004 )
    -------------------------------------------------------------------------
CODE
  Segment part 56. NOT NEEDED.
    -------------------------------------------------------------------------
DATA_C
  Relative segment, address: CODE_AREA 00001990 - 00001997 (0x8 bytes), align: 2
  Segment part 2.             Intra module refs:   menu_sk
    -------------------------------------------------------------------------
DATA_C
  Relative segment, address: CODE_AREA 00001998 - 0000199F (0x8 bytes), align: 2
  Segment part 3.             Intra module refs:   menu_sk
    -------------------------------------------------------------------------
DATA_C
  Relative segment, address: CODE_AREA 000019A0 - 000019EB (0x4c bytes), align: 2
  Segment part 4.             Intra module refs:   Segment part 14
                                                   UpdateCSMname
                                                   main
           ENTRY                   ADDRESS         REF BY
           =====                   =======         ======
           MAINCSM                 000019B0 
    -------------------------------------------------------------------------
DATA_C
  Relative segment, address: CODE_AREA 000019EC - 00001A03 (0x18 bytes), align: 2
  Segment part 5.             Intra module refs:   read_cfg
    -------------------------------------------------------------------------
DATA_C
  Relative segment, address: CODE_AREA 00001A04 - 00001A1B (0x18 bytes), align: 2
  Segment part 6.             Intra module refs:   save_file
    -------------------------------------------------------------------------
DATA_C
  Relative segment, address: CODE_AREA 00001A1C - 00001A43 (0x28 bytes), align: 2
  Segment part 7.             Intra module refs:   menu_onkey
    -------------------------------------------------------------------------
DATA_C
  Segment part 8. NOT NEEDED.
    -------------------------------------------------------------------------
DATA_C
  Relative segment, address: CODE_AREA 00001A44 - 00001A4B (0x8 bytes), align: 2
  Segment part 9.             Intra module refs:   menu_iconhndl
    -------------------------------------------------------------------------
DATA_C
  Relative segment, address: CODE_AREA 00001A4C - 00001A57 (0xc bytes), align: 2
  Segment part 11.            Intra module refs:   Segment part 14
           ENTRY                   ADDRESS         REF BY
           =====                   =======         ======
           menusoftkeys            00001A4C 
    -------------------------------------------------------------------------
DATA_C
  Relative segment, address: CODE_AREA 00001A58 - 00001A6F (0x18 bytes), align: 2
  Segment part 12.            Intra module refs:   menu_skt
           ENTRY                   ADDRESS         REF BY
           =====                   =======         ======
           menu_sk                 00001A58 
    -------------------------------------------------------------------------
DATA_C
  Relative segment, address: CODE_AREA 00001A70 - 00001A77 (0x8 bytes), align: 2
  Segment part 13.            Intra module refs:   Segment part 14
           ENTRY                   ADDRESS         REF BY
           =====                   =======         ======
           menu_skt                00001A70 
    -------------------------------------------------------------------------
DATA_C
  Relative segment, address: CODE_AREA 00001A78 - 00001AB7 (0x40 bytes), align: 2
  Segment part 14.            Intra module refs:   maincsm_oncreate
           ENTRY                   ADDRESS         REF BY
           =====                   =======         ======
           main_menu               00001A8C 
           menuheader              00001A78 
    -------------------------------------------------------------------------
DATA_C
  Relative segment, address: CODE_AREA 00001AB8 - 00001ABB (0x4 bytes), align: 2
  Segment part 15.            Intra module refs:   MAINCSM
           ENTRY                   ADDRESS         REF BY
           =====                   =======         ======
           minus11                 00001AB8 
    -------------------------------------------------------------------------
DATA_C
  Relative segment, address: CODE_AREA 00001ABC - 00001BD3 (0x118 bytes), align: 2
  Segment part 16.            Intra module refs:   MAINCSM
           ENTRY                   ADDRESS         REF BY
           =====                   =======         ======
           maincsm_name_body       00001ABC 
    -------------------------------------------------------------------------
CODE
  Relative segment, address: CODE_AREA 00000D5C - 00000D77 (0x1c bytes), align: 2
  Segment part 57.            Intra module refs:   main
           ENTRY                   ADDRESS         REF BY
           =====                   =======         ======
           UpdateCSMname           00000D5C 
               stack 1 = 00000000 ( 00000004 )
    -------------------------------------------------------------------------
CODE
  Segment part 58. NOT NEEDED.
    -------------------------------------------------------------------------
CODE
  Relative segment, address: CODE_AREA 00000D78 - 00000DAB (0x34 bytes), align: 2
  Segment part 59.
           ENTRY                   ADDRESS         REF BY
           =====                   =======         ======
           main                    00000D78        Absolute parts (?ABS_ENTRY_MOD)
               stack 1 = 00000000 ( 00000030 )
    -------------------------------------------------------------------------
CODE
  Segment part 60. NOT NEEDED.Intra module refs:   menu_onkey
    -------------------------------------------------------------------------
CODE
  Segment part 61. NOT NEEDED.Intra module refs:   menu_onkey
    -------------------------------------------------------------------------
CODE
  Segment part 62. NOT NEEDED.Intra module refs:   Killer
    -------------------------------------------------------------------------
CSTACK
  Segment part 1. NOT NEEDED.
    -------------------------------------------------------------------------
INITTAB
  Relative segment, address: CODE_AREA 00001D7C - 00001D87 (0xc bytes), align: 2
  Segment part 63. ROOT.
           ENTRY                   ADDRESS         REF BY
           =====                   =======         ======
           ?init?tab?DATA_Z        00001D7C 

    *************************************************************************

  FILE NAME : D:\Pasha\elf\googlecode\MyMenu2\MyMenu2_Editor\Release\Obj\open_select_file.r79
  PROGRAM MODULE, NAME : open_select_file

  SEGMENTS IN THE MODULE
  ======================
DATA_Z
  Relative segment, address: CODE_AREA 00001DA8 - 00001DAB (0x4 bytes), align: 2
  Segment part 9.             Intra module refs:   Segment part 28
           ENTRY                   ADDRESS         REF BY
           =====                   =======         ======
           fltop                   00001DA8 
    -------------------------------------------------------------------------
CODE
  Segment part 18. NOT NEEDED.
    -------------------------------------------------------------------------
CODE
  Relative segment, address: CODE_AREA 00000DAC - 00000DE7 (0x3c bytes), align: 2
  Segment part 19.            Intra module refs:   CreateRootMenu
                                                   FindFiles
                                                   filelist_menu_ghook
           ENTRY                   ADDRESS         REF BY
           =====                   =======         ======
           Free_FLIST              00000DAC 
               stack 1 = 00000000 ( 00000008 )
    -------------------------------------------------------------------------
CODE
  Segment part 20. NOT NEEDED.
    -------------------------------------------------------------------------
DATA_C
  Relative segment, address: CODE_AREA 00001BD4 - 00001BDB (0x8 bytes), align: 2
  Segment part 2.             Intra module refs:   Segment part 15
    -------------------------------------------------------------------------
DATA_C
  Relative segment, address: CODE_AREA 00001BDC - 00001BE3 (0x8 bytes), align: 2
  Segment part 3.             Intra module refs:   Segment part 15
    -------------------------------------------------------------------------
DATA_C
  Relative segment, address: CODE_AREA 00001D68 - 00001D69 (0x2 bytes), align: 0
  Segment part 4.             Intra module refs:   Segment part 15
    -------------------------------------------------------------------------
DATA_C
  Relative segment, address: CODE_AREA 00001BE4 - 00001BEF (0xc bytes), align: 2
  Segment part 5.             Intra module refs:   FindFiles
                                                   filelist_menu_onkey
           ENTRY                   ADDRESS         REF BY
           =====                   =======         ======
           back                    00001BE4 
    -------------------------------------------------------------------------
DATA_C
  Segment part 6. NOT NEEDED.
    -------------------------------------------------------------------------
DATA_C
  Relative segment, address: CODE_AREA 00001BF0 - 00001BF7 (0x8 bytes), align: 2
  Segment part 7.             Intra module refs:   filelist_menu_iconhndl
    -------------------------------------------------------------------------
DATA_C
  Relative segment, address: CODE_AREA 00001BF8 - 00001BFF (0x8 bytes), align: 2
  Segment part 8.             Intra module refs:   CreateRootMenu
    -------------------------------------------------------------------------
CODE
  Relative segment, address: CODE_AREA 00000DE8 - 00000E17 (0x30 bytes), align: 2
  Segment part 21.            Intra module refs:   AddToFList
           ENTRY                   ADDRESS         REF BY
           =====                   =======         ======
           strcmp_nocase           00000DE8 
    -------------------------------------------------------------------------
CODE
  Segment part 22. NOT NEEDED.
    -------------------------------------------------------------------------
CODE
  Relative segment, address: CODE_AREA 00000E18 - 00000EC7 (0xb0 bytes), align: 2
  Segment part 23.            Intra module refs:   CreateRootMenu
                                                   FindFiles
           ENTRY                   ADDRESS         REF BY
           =====                   =======         ======
           AddToFList              00000E18 
               stack 1 = 00000000 ( 00000018 )
    -------------------------------------------------------------------------
CODE
  Segment part 24. NOT NEEDED.
    -------------------------------------------------------------------------
CODE
  Relative segment, address: CODE_AREA 00000EC8 - 0000105B (0x194 bytes), align: 2
  Segment part 25.            Intra module refs:   filelist_menu_onkey
                                                   open_select_file_gui
           ENTRY                   ADDRESS         REF BY
           =====                   =======         ======
           FindFiles               00000EC8 
               stack 1 = 00000000 ( 000004E4 )
    -------------------------------------------------------------------------
CODE
  Segment part 26. NOT NEEDED.
    -------------------------------------------------------------------------
CODE
  Relative segment, address: CODE_AREA 0000105C - 0000109F (0x44 bytes), align: 2
  Segment part 27.            Intra module refs:   FindFLISTtByN
           ENTRY                   ADDRESS         REF BY
           =====                   =======         ======
           FindFLISTtByNS          0000105C 
    -------------------------------------------------------------------------
CODE
  Relative segment, address: CODE_AREA 000010A0 - 000010A3 (0x4 bytes), align: 2
  Segment part 28.            Intra module refs:   AddToFList
                                                   FindFLISTtByNS
                                                   Free_FLIST
    -------------------------------------------------------------------------
CODE
  Segment part 29. NOT NEEDED.
    -------------------------------------------------------------------------
CODE
  Relative segment, address: CODE_AREA 000010A4 - 000010F7 (0x54 bytes), align: 2
  Segment part 30.            Intra module refs:   filelist_menu_iconhndl
                                                   filelist_menu_onkey
           ENTRY                   ADDRESS         REF BY
           =====                   =======         ======
           FindFLISTtByN           000010A4 
               stack 1 = 00000000 ( 00000008 )
    -------------------------------------------------------------------------
CODE
  Segment part 31. NOT NEEDED.
    -------------------------------------------------------------------------
CODE
  Relative segment, address: CODE_AREA 000010F8 - 00001143 (0x4c bytes), align: 2
  Segment part 32.            Intra module refs:   filelist_menu_onkey
           ENTRY                   ADDRESS         REF BY
           =====                   =======         ======
           SavePath                000010F8 
               stack 1 = 00000000 ( 0000003C )
    -------------------------------------------------------------------------
CODE
  Segment part 33. NOT NEEDED.
    -------------------------------------------------------------------------
CODE
  Relative segment, address: CODE_AREA 00001144 - 00001243 (0x100 bytes), align: 2
  Segment part 34.            Intra module refs:   Segment part 11
           ENTRY                   ADDRESS         REF BY
           =====                   =======         ======
           filelist_menu_onkey     00001144 
               stack 1 = 00000000 ( 00000014 )
    -------------------------------------------------------------------------
CODE
  Segment part 35. NOT NEEDED.
    -------------------------------------------------------------------------
CODE
  Relative segment, address: CODE_AREA 00001244 - 0000127B (0x38 bytes), align: 2
  Segment part 36.            Intra module refs:   Segment part 11
           ENTRY                   ADDRESS         REF BY
           =====                   =======         ======
           filelist_menu_ghook     00001244 
               stack 1 = 00000000 ( 0000000C )
    -------------------------------------------------------------------------
CODE
  Segment part 37. NOT NEEDED.
    -------------------------------------------------------------------------
CODE
  Relative segment, address: CODE_AREA 0000127C - 00001353 (0xd8 bytes), align: 2
  Segment part 38.            Intra module refs:   Segment part 11
           ENTRY                   ADDRESS         REF BY
           =====                   =======         ======
           filelist_menu_iconhndl
                                   0000127C 
               stack 1 = 00000000 ( 0000001C )
    -------------------------------------------------------------------------
CODE
  Segment part 39. NOT NEEDED.
    -------------------------------------------------------------------------
DATA_I
  Relative segment, address: DATA_AREA 00000038 - 000000F7 (0xc0 bytes), align: 2
  Segment part 10.            Intra module refs:   CreateRootMenu
                                                   Segment part 11
                                                   filelist_menu_onkey
                                                   open_select_file_gui
           ENTRY                   ADDRESS         REF BY
           =====                   =======         ======
           filelist_HDR            00000038 
           filelist_STRUCT         000000CC 
           header                  0000004C 
    -------------------------------------------------------------------------
DATA_I
  Relative segment, address: DATA_AREA 000000F8 - 00000103 (0xc bytes), align: 2
  Segment part 12.            Intra module refs:   Segment part 11
           ENTRY                   ADDRESS         REF BY
           =====                   =======         ======
           fmenusoftkeys           000000F8 
    -------------------------------------------------------------------------
DATA_I
  Relative segment, address: DATA_AREA 00000104 - 0000011B (0x18 bytes), align: 2
  Segment part 14.            Intra module refs:   Segment part 17
           ENTRY                   ADDRESS         REF BY
           =====                   =======         ======
           fmenu_sk                00000104 
    -------------------------------------------------------------------------
DATA_I
  Relative segment, address: DATA_AREA 0000011C - 00000123 (0x8 bytes), align: 2
  Segment part 16.            Intra module refs:   Segment part 11
           ENTRY                   ADDRESS         REF BY
           =====                   =======         ======
           fmenu_skt               0000011C 
    -------------------------------------------------------------------------
CODE
  Relative segment, address: CODE_AREA 00001354 - 000013DB (0x88 bytes), align: 2
  Segment part 40.            Intra module refs:   filelist_menu_onkey
                                                   open_select_file_gui
           ENTRY                   ADDRESS         REF BY
           =====                   =======         ======
           CreateRootMenu          00001354 
               stack 1 = 00000000 ( 00000030 )
    -------------------------------------------------------------------------
CODE
  Segment part 41. NOT NEEDED.
    -------------------------------------------------------------------------
CODE
  Relative segment, address: CODE_AREA 000013DC - 000014EF (0x114 bytes), align: 2
  Segment part 42.
           ENTRY                   ADDRESS         REF BY
           =====                   =======         ======
           open_select_file_gui    000013DC        on_exmenu (ed_gui)
               stack 1 = 00000000 ( 000000D4 )
    -------------------------------------------------------------------------
CSTACK
  Segment part 1. NOT NEEDED.
    -------------------------------------------------------------------------
DATA_ID
  Relative segment, address: CODE_AREA 00000038 - 000000F7 (0xc0 bytes), align: 2
  Segment part 11.            Intra module refs:   Segment part 10
    -------------------------------------------------------------------------
DATA_ID
  Relative segment, address: CODE_AREA 000000F8 - 00000103 (0xc bytes), align: 2
  Segment part 13.            Intra module refs:   fmenusoftkeys
    -------------------------------------------------------------------------
DATA_ID
  Relative segment, address: CODE_AREA 00000104 - 0000011B (0x18 bytes), align: 2
  Segment part 15.            Intra module refs:   fmenu_sk
    -------------------------------------------------------------------------
DATA_ID
  Relative segment, address: CODE_AREA 0000011C - 00000123 (0x8 bytes), align: 2
  Segment part 17.            Intra module refs:   fmenu_skt
    -------------------------------------------------------------------------
DATA_ID
  Segment part 43. TENTATIVE. Used definition from ed_gui
           ENTRY                   ADDRESS         REF BY
           =====                   =======         ======
           ?*?DATA_ID              
    -------------------------------------------------------------------------
INITTAB
  Segment part 44. TENTATIVE. Used definition from ed_gui
           ENTRY                   ADDRESS         REF BY
           =====                   =======         ======
           ?init?tab?DATA_I        
    -------------------------------------------------------------------------
INITTAB
  Segment part 45. TENTATIVE. Used definition from main
           ENTRY                   ADDRESS         REF BY
           =====                   =======         ======
           ?init?tab?DATA_Z        

    *************************************************************************

  FILE NAME : D:\Pasha\elf\googlecode\MyMenu2\MyMenu2_Editor\Release\Obj\option_menu.r79
  PROGRAM MODULE, NAME : option_menu

  SEGMENTS IN THE MODULE
  ======================
DATA_C
  Relative segment, address: CODE_AREA 00001C00 - 00001C07 (0x8 bytes), align: 2
  Segment part 2.             Intra module refs:   mmenu_sk
    -------------------------------------------------------------------------
DATA_C
  Relative segment, address: CODE_AREA 00001C08 - 00001C0F (0x8 bytes), align: 2
  Segment part 3.             Intra module refs:   mmenu_sk
    -------------------------------------------------------------------------
DATA_C
  Relative segment, address: CODE_AREA 00001C10 - 00001C17 (0x8 bytes), align: 2
  Segment part 4.             Intra module refs:   Segment part 14
    -------------------------------------------------------------------------
DATA_C
  Relative segment, address: CODE_AREA 00001C18 - 00001C1F (0x8 bytes), align: 2
  Segment part 5.             Intra module refs:   option_menu_ITEMS
    -------------------------------------------------------------------------
DATA_C
  Relative segment, address: CODE_AREA 00001C20 - 00001C23 (0x4 bytes), align: 2
  Segment part 6.             Intra module refs:   option_menu_ITEMS
    -------------------------------------------------------------------------
DATA_C
  Relative segment, address: CODE_AREA 00001C24 - 00001C2B (0x8 bytes), align: 2
  Segment part 7.             Intra module refs:   option_menu_ITEMS
    -------------------------------------------------------------------------
DATA_C
  Relative segment, address: CODE_AREA 00001C2C - 00001C33 (0x8 bytes), align: 2
  Segment part 8.             Intra module refs:   option_menu_ITEMS
    -------------------------------------------------------------------------
DATA_C
  Relative segment, address: CODE_AREA 00001D6A - 00001D6C (0x3 bytes), align: 0
  Segment part 9.             Intra module refs:   option_menu_ITEMS
    -------------------------------------------------------------------------
DATA_C
  Relative segment, address: CODE_AREA 00001C34 - 00001C3B (0x8 bytes), align: 2
  Segment part 10.            Intra module refs:   option_menu_ITEMS
    -------------------------------------------------------------------------
DATA_C
  Relative segment, address: CODE_AREA 00001C3C - 00001C47 (0xc bytes), align: 2
  Segment part 11.            Intra module refs:   Segment part 14
           ENTRY                   ADDRESS         REF BY
           =====                   =======         ======
           mmenusoftkeys           00001C3C 
    -------------------------------------------------------------------------
DATA_C
  Relative segment, address: CODE_AREA 00001C48 - 00001C5F (0x18 bytes), align: 2
  Segment part 12.            Intra module refs:   mmenu_skt
           ENTRY                   ADDRESS         REF BY
           =====                   =======         ======
           mmenu_sk                00001C48 
    -------------------------------------------------------------------------
DATA_C
  Relative segment, address: CODE_AREA 00001C60 - 00001C67 (0x8 bytes), align: 2
  Segment part 13.            Intra module refs:   Segment part 14
           ENTRY                   ADDRESS         REF BY
           =====                   =======         ======
           mmenu_skt               00001C60 
    -------------------------------------------------------------------------
CODE
  Segment part 17. NOT NEEDED.
    -------------------------------------------------------------------------
CODE
  Relative segment, address: CODE_AREA 000014F0 - 000014F7 (0x8 bytes), align: 2
  Segment part 18.            Intra module refs:   Segment part 14
           ENTRY                   ADDRESS         REF BY
           =====                   =======         ======
           option_menu_keyhook     000014F0 
    -------------------------------------------------------------------------
CODE
  Segment part 19. NOT NEEDED.
    -------------------------------------------------------------------------
CODE
  Relative segment, address: CODE_AREA 000014F8 - 0000150B (0x14 bytes), align: 2
  Segment part 20.            Intra module refs:   Segment part 14
           ENTRY                   ADDRESS         REF BY
           =====                   =======         ======
           option_menu_ghook       000014F8 
               stack 1 = 00000000 ( 00000004 )
    -------------------------------------------------------------------------
CODE
  Segment part 21. NOT NEEDED.
    -------------------------------------------------------------------------
CODE
  Relative segment, address: CODE_AREA 0000150C - 00001527 (0x1c bytes), align: 2
  Segment part 22.            Intra module refs:   option_menu_HNDLS
           ENTRY                   ADDRESS         REF BY
           =====                   =======         ======
           menu_edit               0000150C 
               stack 1 = 00000000 ( 00000004 )
    -------------------------------------------------------------------------
CODE
  Segment part 23. NOT NEEDED.
    -------------------------------------------------------------------------
CODE
  Relative segment, address: CODE_AREA 00001528 - 000015CF (0xa8 bytes), align: 2
  Segment part 24.            Intra module refs:   option_menu_HNDLS
           ENTRY                   ADDRESS         REF BY
           =====                   =======         ======
           menu_add                00001528 
               stack 1 = 00000000 ( 0000000C )
    -------------------------------------------------------------------------
CODE
  Segment part 25. NOT NEEDED.
    -------------------------------------------------------------------------
CODE
  Relative segment, address: CODE_AREA 000015D0 - 000016A7 (0xd8 bytes), align: 2
  Segment part 26.            Intra module refs:   option_menu_HNDLS
           ENTRY                   ADDRESS         REF BY
           =====                   =======         ======
           menu_insert             000015D0 
               stack 1 = 00000000 ( 0000000C )
    -------------------------------------------------------------------------
CODE
  Segment part 27. NOT NEEDED.
    -------------------------------------------------------------------------
CODE
  Relative segment, address: CODE_AREA 000016A8 - 0000178B (0xe4 bytes), align: 2
  Segment part 28.            Intra module refs:   option_menu_HNDLS
           ENTRY                   ADDRESS         REF BY
           =====                   =======         ======
           menu_del                000016A8 
               stack 1 = 00000000 ( 00000010 )
    -------------------------------------------------------------------------
CODE
  Relative segment, address: CODE_AREA 0000178C - 0000178F (0x4 bytes), align: 2
  Segment part 29.            Intra module refs:   menu_add
                                                   menu_del
                                                   menu_insert
    -------------------------------------------------------------------------
CODE
  Segment part 30. NOT NEEDED.
    -------------------------------------------------------------------------
CODE
  Relative segment, address: CODE_AREA 00001790 - 0000181F (0x90 bytes), align: 2
  Segment part 31.            Intra module refs:   option_menu_HNDLS
           ENTRY                   ADDRESS         REF BY
           =====                   =======         ======
           menu_moveup             00001790 
               stack 1 = 00000000 ( 00000004 )
    -------------------------------------------------------------------------
CODE
  Segment part 32. NOT NEEDED.
    -------------------------------------------------------------------------
CODE
  Relative segment, address: CODE_AREA 00001820 - 000018B7 (0x98 bytes), align: 2
  Segment part 33.            Intra module refs:   option_menu_HNDLS
           ENTRY                   ADDRESS         REF BY
           =====                   =======         ======
           menu_movedown           00001820 
               stack 1 = 00000000 ( 00000008 )
    -------------------------------------------------------------------------
CODE
  Relative segment, address: CODE_AREA 000018B8 - 000018BB (0x4 bytes), align: 2
  Segment part 34.            Intra module refs:   menu_del
                                                   menu_edit
                                                   menu_insert
                                                   menu_movedown
                                                   menu_moveup
    -------------------------------------------------------------------------
CODE
  Relative segment, address: CODE_AREA 000018BC - 000018BF (0x4 bytes), align: 2
  Segment part 35.            Intra module refs:   menu_add
                                                   menu_del
                                                   menu_insert
                                                   menu_movedown
                                                   menu_moveup
    -------------------------------------------------------------------------
CODE
  Relative segment, address: CODE_AREA 000018C0 - 000018C3 (0x4 bytes), align: 2
  Segment part 36.            Intra module refs:   menu_del
                                                   menu_movedown
                                                   menu_moveup
    -------------------------------------------------------------------------
CODE
  Segment part 37. NOT NEEDED.
    -------------------------------------------------------------------------
DATA_C
  Relative segment, address: CODE_AREA 00001C68 - 00001CA7 (0x40 bytes), align: 2
  Segment part 14.            Intra module refs:   show_option_menu
           ENTRY                   ADDRESS         REF BY
           =====                   =======         ======
           option_menu             00001C7C 
           option_menu_header      00001C68 
    -------------------------------------------------------------------------
DATA_C
  Relative segment, address: CODE_AREA 00001CA8 - 00001CBF (0x18 bytes), align: 2
  Segment part 15.            Intra module refs:   Segment part 14
           ENTRY                   ADDRESS         REF BY
           =====                   =======         ======
           option_menu_HNDLS       00001CA8 
    -------------------------------------------------------------------------
DATA_C
  Relative segment, address: CODE_AREA 00001CC0 - 00001D67 (0xa8 bytes), align: 2
  Segment part 16.            Intra module refs:   Segment part 14
           ENTRY                   ADDRESS         REF BY
           =====                   =======         ======
           option_menu_ITEMS       00001CC0 
    -------------------------------------------------------------------------
CODE
  Relative segment, address: CODE_AREA 000018C4 - 00001927 (0x64 bytes), align: 2
  Segment part 38.
           ENTRY                   ADDRESS         REF BY
           =====                   =======         ======
           show_option_menu        000018C4        menu_onkey (main)
               stack 1 = 00000000 ( 00000018 )
    -------------------------------------------------------------------------
CODE
  Segment part 39. NOT NEEDED.Intra module refs:   menu_add
                                                   menu_edit
                                                   menu_insert
    -------------------------------------------------------------------------
CODE
  Segment part 40. NOT NEEDED.Intra module refs:   menu_del
                                                   menu_movedown
                                                   menu_moveup
    -------------------------------------------------------------------------
CSTACK
  Segment part 1. NOT NEEDED.




                ****************************************
                *                                      *
                *            MODULE SUMMARY            *
                *                                      *
                ****************************************

Module             CODE   DATA
------             ----   ----
                  (Rel)  (Rel)
ed_gui            1 036     56
  + shared           12
func                  8
main              2 936
  + shared           12
open_select_file  2 146    236
option_menu       1 443
N/A (alignment)
------            -----    ---
Total:            7 593    292


                ****************************************
                *                                      *
                *              CALL GRAPH              *
                *                                      *
                ****************************************

  ->Sub-tree of type: Indirectly called function tree that does not make
                    : indirect calls (Is not an interrupt and is not flagged
                    : as not overlayable)
                             CSTACK
    | Stack used (prev) :  00000000
  01  on_exmenu
      | Stack used (prev) :  00000000
      | + function block  :  00000008
  <-Sub-tree of type: Indirectly called function tree that does not make
                    : indirect calls (Is not an interrupt and is not flagged
                    : as not overlayable)
    | Stack used          :  00000008


  ->Sub-tree of type: Indirectly called function tree that does not make
                    : indirect calls (Is not an interrupt and is not flagged
                    : as not overlayable)
                             CSTACK
    | Stack used (prev) :  00000000
  01  ed_onkey
      | Stack used (prev) :  00000000
      | + function block  :  0000000C
  <-Sub-tree of type: Indirectly called function tree that does not make
                    : indirect calls (Is not an interrupt and is not flagged
                    : as not overlayable)
    | Stack used          :  0000000C


  ->Sub-tree of type: Indirectly called function tree that does not make
                    : indirect calls (Is not an interrupt and is not flagged
                    : as not overlayable)
                             CSTACK
    | Stack used (prev) :  00000000
  01  ed_ghook
      | Stack used (prev) :  00000000
      | + function block  :  00000034
  <-Sub-tree of type: Indirectly called function tree that does not make
                    : indirect calls (Is not an interrupt and is not flagged
                    : as not overlayable)
    | Stack used          :  00000034


  ->Sub-tree of type: Indirectly called function tree that does not make
                    : indirect calls (Is not an interrupt and is not flagged
                    : as not overlayable)
                             CSTACK
    | Stack used (prev) :  00000000
  01  ed_locret
      | Stack used (prev) :  00000000
      | + function block  :  00000000
  <-Sub-tree of type: Indirectly called function tree that does not make
                    : indirect calls (Is not an interrupt and is not flagged
                    : as not overlayable)
    | Stack used          :  00000000


  ->Sub-tree of type: Indirectly called function tree that does not make
                    : indirect calls (Is not an interrupt and is not flagged
                    : as not overlayable)
                             CSTACK
    | Stack used (prev) :  00000000
  01  menu_onkey
      | Stack used (prev) :  00000000
      | + function block  :  00000008
  <-Sub-tree of type: Indirectly called function tree that does not make
                    : indirect calls (Is not an interrupt and is not flagged
                    : as not overlayable)
    | Stack used          :  00000008


  ->Sub-tree of type: Indirectly called function tree that does not make
                    : indirect calls (Is not an interrupt and is not flagged
                    : as not overlayable)
                             CSTACK
    | Stack used (prev) :  00000000
  01  menu_ghook
      | Stack used (prev) :  00000000
      | + function block  :  00000004
  <-Sub-tree of type: Indirectly called function tree that does not make
                    : indirect calls (Is not an interrupt and is not flagged
                    : as not overlayable)
    | Stack used          :  00000004


  ->Sub-tree of type: Indirectly called function tree that does not make
                    : indirect calls (Is not an interrupt and is not flagged
                    : as not overlayable)
                             CSTACK
    | Stack used (prev) :  00000000
  01  menu_iconhndl
      | Stack used (prev) :  00000000
      | + function block  :  00000018
  <-Sub-tree of type: Indirectly called function tree that does not make
                    : indirect calls (Is not an interrupt and is not flagged
                    : as not overlayable)
    | Stack used          :  00000018


  ->Sub-tree of type: Indirectly called function tree that does not make
                    : indirect calls (Is not an interrupt and is not flagged
                    : as not overlayable)
                             CSTACK
    | Stack used (prev) :  00000000
  01  maincsm_oncreate
      | Stack used (prev) :  00000000
      | + function block  :  00000020
  <-Sub-tree of type: Indirectly called function tree that does not make
                    : indirect calls (Is not an interrupt and is not flagged
                    : as not overlayable)
    | Stack used          :  00000020


  ->Sub-tree of type: Indirectly called function tree that does not make
                    : indirect calls (Is not an interrupt and is not flagged
                    : as not overlayable)
                             CSTACK
    | Stack used (prev) :  00000000
  01  maincsm_onmessage
      | Stack used (prev) :  00000000
      | + function block  :  0000000C
  <-Sub-tree of type: Indirectly called function tree that does not make
                    : indirect calls (Is not an interrupt and is not flagged
                    : as not overlayable)
    | Stack used          :  0000000C


  ->Sub-tree of type: Indirectly called function tree that does not make
                    : indirect calls (Is not an interrupt and is not flagged
                    : as not overlayable)
                             CSTACK
    | Stack used (prev) :  00000000
  01  Killer
      | Stack used (prev) :  00000000
      | + function block  :  00000008
  <-Sub-tree of type: Indirectly called function tree that does not make
                    : indirect calls (Is not an interrupt and is not flagged
                    : as not overlayable)
    | Stack used          :  00000008


  ->Sub-tree of type: Indirectly called function tree that does not make
                    : indirect calls (Is not an interrupt and is not flagged
                    : as not overlayable)
                             CSTACK
    | Stack used (prev) :  00000000
  01  maincsm_onclose
      | Stack used (prev) :  00000000
      | + function block  :  00000004
  <-Sub-tree of type: Indirectly called function tree that does not make
                    : indirect calls (Is not an interrupt and is not flagged
                    : as not overlayable)
    | Stack used          :  00000004


  ->Sub-tree of type: Indirectly called function tree that does not make
                    : indirect calls (Is not an interrupt and is not flagged
                    : as not overlayable)
                             CSTACK
    | Stack used (prev) :  00000000
  01  filelist_menu_onkey
      | Stack used (prev) :  00000000
      | + function block  :  00000014
  <-Sub-tree of type: Indirectly called function tree that does not make
                    : indirect calls (Is not an interrupt and is not flagged
                    : as not overlayable)
    | Stack used          :  00000014


  ->Sub-tree of type: Indirectly called function tree that does not make
                    : indirect calls (Is not an interrupt and is not flagged
                    : as not overlayable)
                             CSTACK
    | Stack used (prev) :  00000000
  01  filelist_menu_ghook
      | Stack used (prev) :  00000000
      | + function block  :  0000000C
  <-Sub-tree of type: Indirectly called function tree that does not make
                    : indirect calls (Is not an interrupt and is not flagged
                    : as not overlayable)
    | Stack used          :  0000000C


  ->Sub-tree of type: Indirectly called function tree that does not make
                    : indirect calls (Is not an interrupt and is not flagged
                    : as not overlayable)
                             CSTACK
    | Stack used (prev) :  00000000
  01  filelist_menu_iconhndl
      | Stack used (prev) :  00000000
      | + function block  :  0000001C
  <-Sub-tree of type: Indirectly called function tree that does not make
                    : indirect calls (Is not an interrupt and is not flagged
                    : as not overlayable)
    | Stack used          :  0000001C


  ->Sub-tree of type: Indirectly called function tree that does not make
                    : indirect calls (Is not an interrupt and is not flagged
                    : as not overlayable)
                             CSTACK
    | Stack used (prev) :  00000000
  01  option_menu_keyhook
      | Stack used (prev) :  00000000
      | + function block  :  00000000
  <-Sub-tree of type: Indirectly called function tree that does not make
                    : indirect calls (Is not an interrupt and is not flagged
                    : as not overlayable)
    | Stack used          :  00000000


  ->Sub-tree of type: Indirectly called function tree that does not make
                    : indirect calls (Is not an interrupt and is not flagged
                    : as not overlayable)
                             CSTACK
    | Stack used (prev) :  00000000
  01  option_menu_ghook
      | Stack used (prev) :  00000000
      | + function block  :  00000004
  <-Sub-tree of type: Indirectly called function tree that does not make
                    : indirect calls (Is not an interrupt and is not flagged
                    : as not overlayable)
    | Stack used          :  00000004


  ->Sub-tree of type: Indirectly called function tree that does not make
                    : indirect calls (Is not an interrupt and is not flagged
                    : as not overlayable)
                             CSTACK
    | Stack used (prev) :  00000000
  01  menu_edit
      | Stack used (prev) :  00000000
      | + function block  :  00000004
  <-Sub-tree of type: Indirectly called function tree that does not make
                    : indirect calls (Is not an interrupt and is not flagged
                    : as not overlayable)
    | Stack used          :  00000004


  ->Sub-tree of type: Indirectly called function tree that does not make
                    : indirect calls (Is not an interrupt and is not flagged
                    : as not overlayable)
                             CSTACK
    | Stack used (prev) :  00000000
  01  menu_add
      | Stack used (prev) :  00000000
      | + function block  :  0000000C
  <-Sub-tree of type: Indirectly called function tree that does not make
                    : indirect calls (Is not an interrupt and is not flagged
                    : as not overlayable)
    | Stack used          :  0000000C


  ->Sub-tree of type: Indirectly called function tree that does not make
                    : indirect calls (Is not an interrupt and is not flagged
                    : as not overlayable)
                             CSTACK
    | Stack used (prev) :  00000000
  01  menu_insert
      | Stack used (prev) :  00000000
      | + function block  :  0000000C
  <-Sub-tree of type: Indirectly called function tree that does not make
                    : indirect calls (Is not an interrupt and is not flagged
                    : as not overlayable)
    | Stack used          :  0000000C


  ->Sub-tree of type: Indirectly called function tree that does not make
                    : indirect calls (Is not an interrupt and is not flagged
                    : as not overlayable)
                             CSTACK
    | Stack used (prev) :  00000000
  01  menu_del
      | Stack used (prev) :  00000000
      | + function block  :  00000010
  <-Sub-tree of type: Indirectly called function tree that does not make
                    : indirect calls (Is not an interrupt and is not flagged
                    : as not overlayable)
    | Stack used          :  00000010


  ->Sub-tree of type: Indirectly called function tree that does not make
                    : indirect calls (Is not an interrupt and is not flagged
                    : as not overlayable)
                             CSTACK
    | Stack used (prev) :  00000000
  01  menu_moveup
      | Stack used (prev) :  00000000
      | + function block  :  00000004
  <-Sub-tree of type: Indirectly called function tree that does not make
                    : indirect calls (Is not an interrupt and is not flagged
                    : as not overlayable)
    | Stack used          :  00000004


  ->Sub-tree of type: Indirectly called function tree that does not make
                    : indirect calls (Is not an interrupt and is not flagged
                    : as not overlayable)
                             CSTACK
    | Stack used (prev) :  00000000
  01  menu_movedown
      | Stack used (prev) :  00000000
      | + function block  :  00000008
  <-Sub-tree of type: Indirectly called function tree that does not make
                    : indirect calls (Is not an interrupt and is not flagged
                    : as not overlayable)
    | Stack used          :  00000008


  ->Sub-tree of type: Function tree
                             CSTACK
    | Stack used (prev) :  00000034
  01  edit_ml
      | Stack used (prev) :  00000034
      | + function block  :  00000060
  <-Sub-tree of type: Function tree
    | Stack used          :  00000094


  ->Sub-tree of type: Function tree
                             CSTACK
    | Stack used (prev) :  00000094
  01  AddtoMenuList
      | Stack used (prev) :  00000094
      | + function block  :  0000001C
  <-Sub-tree of type: Function tree
    | Stack used          :  000000B0


  ->Sub-tree of type: Function tree
                             CSTACK
    | Stack used (prev) :  000000B0
  01  FreeMenuList
      | Stack used (prev) :  000000B0
      | + function block  :  0000000C
  <-Sub-tree of type: Function tree
    | Stack used          :  000000BC


  ->Sub-tree of type: Function tree
                             CSTACK
    | Stack used (prev) :  000000BC
  01  get_mlitem
      | Stack used (prev) :  000000BC
      | + function block  :  00000000
  <-Sub-tree of type: Function tree
    | Stack used          :  000000BC


  ->Sub-tree of type: Function tree
                             CSTACK
    | Stack used (prev) :  000000BC
  01  strchrinline
      | Stack used (prev) :  000000BC
      | + function block  :  00000000
  <-Sub-tree of type: Function tree
    | Stack used          :  000000BC


  ->Sub-tree of type: Function tree
                             CSTACK
    | Stack used (prev) :  000000BC
  01  gotoRealPos
      | Stack used (prev) :  000000BC
      | + function block  :  00000000
  <-Sub-tree of type: Function tree
    | Stack used          :  000000BC


  ->Sub-tree of type: Function tree
                             CSTACK
    | Stack used (prev) :  000000BC
  01  gotoLineEnd
      | Stack used (prev) :  000000BC
      | + function block  :  00000000
  <-Sub-tree of type: Function tree
    | Stack used          :  000000BC


  ->Sub-tree of type: Function tree
                             CSTACK
    | Stack used (prev) :  000000BC
  01  CheckType
      | Stack used (prev) :  000000BC
      | + function block  :  00000004
  <-Sub-tree of type: Function tree
    | Stack used          :  000000C0


  ->Sub-tree of type: Function tree
                             CSTACK
    | Stack used (prev) :  000000C0
  01  read_cfg
      | Stack used (prev) :  000000C0
      | + function block  :  00000048
  <-Sub-tree of type: Function tree
    | Stack used          :  00000108


  ->Sub-tree of type: Function tree
                             CSTACK
    | Stack used (prev) :  00000108
  01  save_file
      | Stack used (prev) :  00000108
      | + function block  :  00000118
  <-Sub-tree of type: Function tree
    | Stack used          :  00000220


  ->Sub-tree of type: Function tree
                             CSTACK
    | Stack used (prev) :  00000220
  01  save_ml
      | Stack used (prev) :  00000220
      | + function block  :  00000014
  <-Sub-tree of type: Function tree
    | Stack used          :  00000234


  ->Sub-tree of type: Function tree
                             CSTACK
    | Stack used (prev) :  00000234
  01  UpdateCSMname
      | Stack used (prev) :  00000234
      | + function block  :  00000004
  <-Sub-tree of type: Function tree
    | Stack used          :  00000238


  ->Sub-tree of type: Function tree
                             CSTACK
    | Stack used (prev) :  00000238
  01  main
      | Stack used (prev) :  00000238
      | + function block  :  00000030
  <-Sub-tree of type: Function tree
    | Stack used          :  00000268


  ->Sub-tree of type: Function tree
                             CSTACK
    | Stack used (prev) :  00000268
  01  Free_FLIST
      | Stack used (prev) :  00000268
      | + function block  :  00000008
  <-Sub-tree of type: Function tree
    | Stack used          :  00000270


  ->Sub-tree of type: Function tree
                             CSTACK
    | Stack used (prev) :  00000270
  01  strcmp_nocase
      | Stack used (prev) :  00000270
      | + function block  :  00000000
  <-Sub-tree of type: Function tree
    | Stack used          :  00000270


  ->Sub-tree of type: Function tree
                             CSTACK
    | Stack used (prev) :  00000270
  01  AddToFList
      | Stack used (prev) :  00000270
      | + function block  :  00000018
  <-Sub-tree of type: Function tree
    | Stack used          :  00000288


  ->Sub-tree of type: Function tree
                             CSTACK
    | Stack used (prev) :  00000288
  01  FindFiles
      | Stack used (prev) :  00000288
      | + function block  :  000004E4
  <-Sub-tree of type: Function tree
    | Stack used          :  0000076C


  ->Sub-tree of type: Function tree
                             CSTACK
    | Stack used (prev) :  0000076C
  01  FindFLISTtByNS
      | Stack used (prev) :  0000076C
      | + function block  :  00000000
  <-Sub-tree of type: Function tree
    | Stack used          :  0000076C


  ->Sub-tree of type: Function tree
                             CSTACK
    | Stack used (prev) :  0000076C
  01  FindFLISTtByN
      | Stack used (prev) :  0000076C
      | + function block  :  00000008
  <-Sub-tree of type: Function tree
    | Stack used          :  00000774


  ->Sub-tree of type: Function tree
                             CSTACK
    | Stack used (prev) :  00000774
  01  SavePath
      | Stack used (prev) :  00000774
      | + function block  :  0000003C
  <-Sub-tree of type: Function tree
    | Stack used          :  000007B0


  ->Sub-tree of type: Function tree
                             CSTACK
    | Stack used (prev) :  000007B0
  01  CreateRootMenu
      | Stack used (prev) :  000007B0
      | + function block  :  00000030
  <-Sub-tree of type: Function tree
    | Stack used          :  000007E0


  ->Sub-tree of type: Function tree
                             CSTACK
    | Stack used (prev) :  000007E0
  01  open_select_file_gui
      | Stack used (prev) :  000007E0
      | + function block  :  000000D4
  <-Sub-tree of type: Function tree
    | Stack used          :  000008B4


  ->Sub-tree of type: Function tree
                             CSTACK
    | Stack used (prev) :  000008B4
  01  show_option_menu
      | Stack used (prev) :  000008B4
      | + function block  :  00000018
  <-Sub-tree of type: Function tree
    | Stack used          :  000008CC




                ****************************************
                *                                      *
                *      SEGMENTS IN ADDRESS ORDER       *
                *                                      *
                ****************************************


SEGMENT              SPACE    START ADDRESS   END ADDRESS     SIZE  TYPE  ALIGN
=======              =====    =============   ===========     ====  ====  =====
ELFBEGIN             CODE_AREA           00000000                     rel    0
DATA_ID              CODE_AREA      00000000 - 00000123         124   rel    2
START                CODE_AREA           00000124                     dse    0
CODE                 CODE_AREA      00000124 - 00001927        1804   rel    2
DATA_C               CODE_AREA      00001928 - 00001D6C         445   rel    2
INITTAB              CODE_AREA      00001D70 - 00001D87          18   rel    2
DATA_Z               CODE_AREA      00001D88 - 00001DAB          24   rel    2
DATA_I               DATA_AREA      00000000 - 00000123         124   rel    2

                ****************************************
                *                                      *
                *        END OF CROSS REFERENCE        *
                *                                      *
                ****************************************

 7 593 bytes of CODE memory
   292 bytes of DATA memory

Errors: none
Warnings: none

